:100000000010001017010000E9000000EB000000E4
:1000100000000000000000000000000000000000E0
:10002000000000000000000000000000ED000000E3
:100030000000000000000000EF000000F1000000E0
:10004000F3000000F3000000F3000000F3000000E4
:10005000F3000000F3000000F3000000F3000000D4
:10006000F3000000F30000000000000000000000AA
:100070000000000000000000F3000000F30000009A
:10008000F3000000F3000000F3000000F3000000A4
:10009000F3000000810D00004D0B0000F300000094
:1000A000F3000000F9030000F3000000F30000007B
:1000B0000000000000000000F3000000000000004D
:1000C00034330000000000107000000034330000E2
:1000D0000040002000000000700000106C020000D2
:1000E0000040002000000000FEE7FEE7FEE7FEE71C
:1000F000FEE7FEE7002310B5934203D21C585C5084
:100100000433F9E710BD00238B4203D200221A50BA
:100110000433F9E77047C0210F4A0905136810B589
:100120000B430E4C13600E4B9C4206D22068616854
:10013000A268FFF7DFFF0C34F5E70A4B9C4205D2BB
:1001400020686168FFF7DFFF0834F6E700F0C6FDBE
:1001500000F028FDFEE7C04680800440C00000009B
:10016000D8000000E8000000FFFFFFFFFFFFFFFFD7
:10017000FFFFFFFFFFFFFFFFFFFFFFFFFFFFFFFF8F
:10018000FFFFFFFFFFFFFFFFFFFFFFFFFFFFFFFF7F
:10019000FFFFFFFFFFFFFFFFFFFFFFFFFFFFFFFF6F
:1001A000FFFFFFFFFFFFFFFFFFFFFFFFFFFFFFFF5F
:1001B000FFFFFFFFFFFFFFFFFFFFFFFFFFFFFFFF4F
:1001C000FFFFFFFFFFFFFFFFFFFFFFFFFFFFFFFF3F
:1001D000FFFFFFFFFFFFFFFFFFFFFFFFFFFFFFFF2F
:1001E000FFFFFFFFFFFFFFFFFFFFFFFFFFFFFFFF1F
:1001F000FFFFFFFFFFFFFFFFFFFFFFFFFFFFFFFF0F
:10020000FFFFFFFFFFFFFFFFFFFFFFFFFFFFFFFFFE
:10021000FFFFFFFFFFFFFFFFFFFFFFFFFFFFFFFFEE
:10022000FFFFFFFFFFFFFFFFFFFFFFFFFFFFFFFFDE
:10023000FFFFFFFFFFFFFFFFFFFFFFFFFFFFFFFFCE
:10024000FFFFFFFFFFFFFFFFFFFFFFFFFFFFFFFFBE
:10025000FFFFFFFFFFFFFFFFFFFFFFFFFFFFFFFFAE
:10026000FFFFFFFFFFFFFFFFFFFFFFFFFFFFFFFF9E
:10027000FFFFFFFFFFFFFFFFFFFFFFFFFFFFFFFF8E
:10028000FFFFFFFFFFFFFFFFFFFFFFFFFFFFFFFF7E
:10029000FFFFFFFFFFFFFFFFFFFFFFFFFFFFFFFF6E
:1002A000FFFFFFFFFFFFFFFFFFFFFFFFFFFFFFFF5E
:1002B000FFFFFFFFFFFFFFFFFFFFFFFFFFFFFFFF4E
:1002C000FFFFFFFFFFFFFFFFFFFFFFFFFFFFFFFF3E
:1002D000FFFFFFFFFFFFFFFFFFFFFFFFFFFFFFFF2E
:1002E000FFFFFFFFFFFFFFFFFFFFFFFFFFFFFFFF1E
:1002F000FFFFFFFFFFFFFFFFFFFFFFFF7073694E70
:1003000007B5012304480021172200F0E9FE034845
:10031000694600F0A5FD07BD0040044000C0014053
:1003200013B501220E48072100F004FE0C480121FC
:10033000002200F0EBFD0A480721002200F0CBFD6F
:100340000128F8D16B469C1D221C0721044800F0AF
:10035000B7FD03480721002200F0ECFD208816BD00
:1003600000C0014082B00190019B5A1E0192002BF7
:1003700001D0C046F8E702B07047A0230122DB0598
:100380001A725A72DA7280228020920199584000C3
:100390000143995099580018014380209950995869
:1003A000000101439950704701280FD0002802D066
:1003B000022816D01FE00122A023101CDB054840B4
:1003C0001872002917D05A72DA7214E0021CA023A6
:1003D0004A40D2B2DB055A7200290CD01872D8728A
:1003E00009E00122A023101CDB054840D872002937
:1003F00001D01A725A7270470421044808B5036884
:100400000B4201D000F072FF08BDC0460040004022
:1004100038B5114C051C201C00F052FF402000F0A4
:10042000B3FE49220D4B5A6200F0C4FD01230222A3
:1004300080084543236165602368201C13432360C3
:100440000C2100F053FF8022C021054B920449008B
:100450005A501A6038BDC046004000400080044039
:1004600000E100E00121044B1A680A431A60AA2245
:100470009A60553A9A60704700400040AA22024BA9
:100480009A60553A9A60704700400040032A03D1B1
:100490000B8B023A93430B83002070470020704778
:1004A00010B5022A16D10C1C0B4B227B1B68920143
:1004B0001B68A2181A325B6C097D9847237B9A014E
:1004C000A218527FA02A01D19F3AA27403220133BD
:1004D00013402373002010BD50000010F0B5161C0F
:1004E0000C1C99B048220190002106A8029302F04A
:1004F00037FD736802210693B368E068079300F044
:1005000043FB0A210890E06800F03EFB314B324F7C
:1005100015933B6809905B6901985B6806A905AA79
:100520009847051E53D18823069C2C499B008C4676
:10053000E218069272608822079B291C0393634489
:10054000B3609200201C079302F00AFD0221019B78
:1005500023482360059B63601E9B1C60214B5A68E7
:100560008A435A605A680A435A60291C04221E4B67
:1005700000F0B6FD291C1A4805221B4B00F0B0FD07
:100580008022029B1202A360184B0198DA67812334
:10059000E3743B6803215B68154A5D68231CA84728
:1005A000051E10D1012323753B68124A5B68019830
:1005B0005D680221231CA847E122636852021A6188
:1005C0000822051C9A75069B7360079BB360281C64
:1005D00019B0F0BD9D04000050000010E0FDFFFFC9
:1005E00000400440008004400102000004E100E0FB
:1005F0008D040000A1040000F0B5036889B0ED335C
:100600001B78041C002B00D1B1E102208723667BFC
:10061000227B60749B00B24200D17EE10021E15058
:10062000A37BB6019B011933FF33E31801931D1817
:100630000423019AA61993701A3673786B70B378F5
:10064000AB701123EB70F278101CA038062800D98B
:100650004CE102F01BFD490007003E0088008800C5
:1006600013015300A06800F0CFF973793079B179A4
:100670001B02034309041A1C0B1CF17913430906DE
:100680001943A06800F0CAF9737A307AB17A1B0274
:10069000034309041A1C0B1CF17A1343090619437E
:1006A000A06800F04BFAC54E301C02F05DFC311C16
:1006B000021C281D02F050FC301C02F055FC0026E4
:1006C000019B01219B78C018019B9870EE7002205D
:1006D00006E00026A06800F09CF90220311CEE70B4
:1006E000FFF762FE311C01E13C22A3689A610C3ADB
:1006F0001A60CF329A60EF3A1A6031E0FFF710FECD
:100700002871000A6871237B627B02A9073193423A
:1007100000D204339B1AA81D01220B7002F01CFCAE
:10072000A37BE27B04A9934200D204339B1A0B7093
:100730000B7801220133E81D0B7002F00DFC281C20
:10074000211C238B01222B72238B0A301B0A6B7214
:10075000113102F001FC019B019A9B7807339370E1
:100760000021E970C2E0A43A51425141CAB2382195
:10077000A3689961B179C9071DD5602119601AE094
:10078000002803D10B68A07C1B07F9D5002868D18D
:10079000F8234F683B40002A37D0502B16D0582BF7
:1007A0000ED12B78591C2970A1688968E954E8702A
:1007B0003821A3689961EB78112B54D1A168E1E746
:1007C000402B00D0E7E004230B6005E02B78591C98
:1007D0002970A1688968E9542B78B179181F08231A
:1007E000377919407379002909D019020B1C3B4352
:1007F0001B1A012BDCD10421A3689961D8E71B02E5
:100800003B438342D4D1E970D2E7182B13D004D8EC
:10081000082B0CD0102B0AD0C9E0282B0BD0302B82
:1008200000D0B8E0B079400701D52E3B17E0B07991
:10083000400600D4CCE02B78043BF018007A8860A6
:1008400029780131297071793079090201438B428D
:10085000AED1002303E0482B00D0C6E00423EB70A8
:10086000A6E70123EB70EB780121052B3ED0B3798D
:100870009B073BD51022A3681A6037E004AF002124
:10088000381C102202F06CFBF379A0683B70331C1B
:100890000833BB602B1DFB607379391CFB803379F7
:1008A000BB80B3797B7000F041F9A0680268A37C3B
:1008B000120702D5002B03D008E0002BF6D0F9E791
:1008C000391C00F0BBF80028EFD001E001237B8049
:1008D0007379F9885A1A002A05DD019A92789B18D3
:1008E000019A5B1A937001217B88EB70A37C002B2B
:1008F00001D00023A3740322637B00200133134043
:100900006373A37B01331A40A273EB78002B0CD1E5
:1009100000290DD00120011C08E0E25828490132CD
:100920008A4201D8E25003E0E1500121FFF73CFD8B
:10093000E37BA27B9A425BD00121228B0A4257D1F2
:10094000228B9B010A4322831E4AE17C12681068B5
:10095000E218E3181B32FF33FF32DB7E056D20689F
:10096000A8470322E37B01331340E37340E0427C5A
:10097000022A02D1032343743AE0012A04D04373CC
:1009800003738373C3738374012302206374002190
:10099000FFF70AFD2CE0102B09D1B3795B0600D5D7
:1009A00006E7F3795B001343DBB28B6000E7102BA3
:1009B00016D8002B08D1032351E7C046FE300000B3
:1009C000801A060050000010082BE6D0012346E7ED
:1009D000102BE6D004D8002BEDD0082BE1D0F5E7A2
:1009E000382B00D037E7052339E7202BEED135E748
:1009F00009B0F0BD002800D04174704704230028DE
:100A000000D0437C181C704708B5002000F040FB64
:100A100008BD08B5002000F04FFB08BD38B50D1C1F
:100A2000041C00F0FBFA291C02F0CBFA4308C01AA0
:100A30009AB280B22261606138BD000038B5F823F7
:100A40004268051C0C1C1340282B2FD00CD8102BEF
:100A50001FD004D8002B57D0082B1AD058E0182BE1
:100A600024D0202B1DD053E0402B3FD007D8302B73
:100A700017D0382B4CD105234B8037334BE0502B0C
:100A80002CD0582B2AD0482B42D104234B8028331A
:100A900041E0A3885A425A4123785B001343AB607C
:100AA0001AE06378DB0701D402230BE0A388002B54
:100AB0000BD1E388002B05D01B4B1868FFF752FCC5
:100AC0001C2328E063802C2325E0A268013B511CF5
:100AD000A1601278AA60A3803C231CE0E3685A1C42
:100AE000E260AA681A70E388013BE380E288382359
:100AF000012A10D86178890700D40433002A0AD16A
:100B000062801032934306E003234B80293302E0D6
:100B1000012363802B333C225A402A60AB616088FA
:100B2000FF38431E984138BD4C000010FF234B8016
:100B3000C33B83612433036070470000002901D068
:100B4000014B19607047C0464C0000100A4A08B5B6
:100B500093681268D20506D5084A196811401960D1
:100B600099680A409A60064B064A1B6810681B6821
:100B7000DB68984708BDC04600000840FFFFFFDF64
:100B800050000010700000100378002B07D042784E
:100B9000042A02D142798A4202D0C018F4E7181C14
:100BA0007047000070B59AB000F0F8F800F09AF8BD
:100BB0000020012100F0F0F980213B4BC901DA6FE0
:100BC00080200A438021DA67DA6F09050A4309ACFD
:100BD000DA67C00000F0D8FA00214422201C02F09D
:100BE000BFF9324B324E099303232373314B324DFD
:100BF000636080231B01A360304B281C0493304B9F
:100C000004A905932F4B221C0793069300230893F6
:100C100033681B685B68984700280ED103AB0093CC
:100C20008023286804A9221CDB05FFF757FC002855
:100C300003D18022244BD2031A60FFF761FBFFF738
:100C40009CFB0520FFF7E4FBFFF70CFC8020C005B0
:100C5000FFF7DAFE80201D49C005FFF7DFFE012106
:100C60000220FFF7A1FB1A48FFF77CFB33682868D6
:100C70001B6801219B68984703980021FFF7BAFE83
:100C80000398FFF7B9FC0398FFF7B8FE032807D1D4
:100C9000BFF34F8F0F4A104BDA60BFF34F8FFEE761
:100CA000FFF7ECFBECE7C04604800440000008407E
:100CB000500000100040002070000010EC300000D8
:100CC0009C3000000000001000E100E0801A0600E7
:100CD000007701000400FA0500ED00E008B500F01F
:100CE00063F808BD10B51D4C0021201C12221123F1
:100CF00000F0F6F9201C1A4C13220123002100F009
:100D0000EFF9201C00F052FA201C164900F09AFA64
:100D10000323E3607E33A360013B23631249012276
:100D2000403B124800F0E2F98023114901229B0068
:100D3000104800F0DBF90522C521636889001343E0
:100D40000D4A636050580D4B03408020C00103439F
:100D5000535080239B03136010BDC04600400440E5
:100D60000080004007B2010074000010B4000010C1
:100D7000DC000010C800001000E100E0FF00FFFFF1
:100D800008B503480349044A00F045FA08BDC046C7
:100D900000800040B4000010C8000010A02008B57A
:100DA000C00500F05FF908BD73B5202000F0ECF934
:100DB00000230193019BFF2B02DC019B0133F8E729
:100DC000012000F0CBF8802000F0CEF923231A4C4C
:100DD0008020A36000F0D8F90125E368164E2B426D
:100DE000FAD003200221154AB567136983430B43E8
:100DF000136100F0C7F8281C00F0BAF82323802004
:100E00003361400000F0C0F96369DB07FCD5802145
:100E100000240B4A4902D36F0B43D367094AA3004E
:100E2000995CD3185A7808485B88013400F058F967
:100E3000092CF3D173BDC0460080044000C00340BC
:100E40000480044030310000004004400268034B3D
:100E500009061340194301607047C046FFFFFFF8C1
:100E600038B5041C10200D1C00F08EF98021104AAA
:100E70008901D36F0B43D36700230E4AE3602A60D6
:100E80002B716B7100F0E4F807232D7940001D40B1
:100E900080236D049B031D43074B0849C01802F0D3
:100EA00090F80138C0B200022843206038BDC04627
:100EB00004800440801A0600802343000047860017
:100EC000043189000B580020834203DA1B049B0D78
:100ED000138001307047012A0ED0002A07D0022A61
:100EE00011D1006B000C411E8841C0B20CE0006BB8
:100EF0000123C840184007E0006B0831C9B2C84060
:100F00000240D0B200E000207047000008B501297F
:100F10000AD9002A04D0802203681205134302E094
:100F20000268034B13400360FFF790FF08BDC04603
:100F3000FFFFFFF7012A04D18A4003681A430260C9
:100F400008E00268044B134001228A4003600368F2
:100F5000934303607047C046FFFFFFF80022034B36
:100F600018645A6401325A647047C04600800440D5
:100F70000022034B9864DA640132DA647047C04699
:100F8000008004400022034B18675A6701325A67F9
:100F90007047C04600800440054B1A1CC0321060E8
:100FA0000020C83350600130506019607047C0465F
:100FB0000080044008B5074B596A1F23CA05120F69
:100FC0001940054B920001314900D05801F0F9FF5A
:100FD00008BDC0460080044054310000064B1A6C26
:100FE0000323134005D00020012B03D1034B1868C5
:100FF00000E003487047C046008004402C310000E8
:10100000001BB700044B10B59C68FFF7E7FF1F23D8
:1010100023400133584310BD0080044008B50A4BFB
:101020001A6F03231340022B06D0032B07D0012B8A
:1010300008D1FFF7D3FF06E0FFF7BCFF03E0FFF79F
:10104000E1FF00E0014808BD00800440001BB7003C
:1010500008B5FFF7E3FF024B996F01F0B2FF08BD3F
:10106000008004404021024AD36F0B43D36770478E
:1010700004800440012907D11C235843034B18184E
:101080000269137D042BFCD07047C0465400001049
:101090001C2330B558430649064C0B181D79012313
:1010A000AB40E26F13436C22E36743589A6130BD53
:1010B00054000010048004401C2358437C21064A3D
:1010C0008358101801229961007904498240CB6F3E
:1010D0009343CB677047C04654000010048004401F
:1010E000002900D01832920013507047436000234B
:1010F000016082600361C36001207047F8B5041C81
:10110000C268076863680069121A00209A420FDA01
:101110000D1CE068591E01F054FFA6687143321C93
:101120007818291C01F018FF0120E3680133E360FF
:10113000F8BDF8B5C2680369041C076800209A422C
:1011400010D063680D1C2069591E01F03AFFA66893
:10115000281C7143321C791801F0FEFE012023691E
:1011600001332361F8BD00008E22054992008B589F
:101170001843044B1840E8231B021843885070475B
:1011800000800440FF0500008E2110B5054C890049
:101190006358054A134002409343E8221202134366
:1011A000635010BD00800440FF05000010B580248E
:1011B000074B6401191DCA6F98332243CA67012285
:1011C0001A6007238360043BC3600D33836210BD44
:1011D0000080044037B5041C0D1C6369DB0707D58C
:1011E0006A462368D11D281C0B70FFF787FFF4E7C0
:1011F00037BD73B5051C0E1C6B699B060AD56B4683
:10120000DC1D301C211CFFF794FF002802D023783E
:101210002B60F1E773BDF8B502264368041C0D1C72
:10122000171C334209D0111CFFF7E3FFFA683B6932
:101230009A4202D16368B3436360291C201CFFF704
:10124000C9FFF8BDF7B50D01061CFFF7E7FE291C25
:10125000071C01F0B6FE00200C1E844206D0281C9C
:1012600001F0AFFE00240C23834264410F23184099
:101270000190281C0199604301F0A3FE4119381C1C
:1012800001F09FFE8022F368011C1343F360FF23EB
:10129000051C19403160010A0B407360F36820019E
:1012A0009343F360019B01991B012343B36268439D
:1012B00001F087FE2D014119381C01F082FEFEBDB0
:1012C0008021074A0902D36F0B43D36700230360D1
:1012D000FF334360034B4361034B83617047C04658
:1012E00004800440FFFF0000FFFFFF004B0703D511
:1012F0001B230268134003600822114202D00368D6
:1013000013430360704700007047C0467047C046F3
:10131000027B3F23510088180001D430FF309843EE
:101320008030704700B58C235A0083581B6A00290F
:1013300004D1196804480840186000BD196880226B
:10134000500208431860F8E7FFFFFEFF00B58C234A
:10135000EE215A00435A8258990704D5126A02486E
:1013600011680840106000BDFFFFFDFF00B58C2331
:101370005A0083581B6A002905D1186880218A0009
:1013800002431A6000BD1968014808401860F9E777
:10139000FFFDFFFF8C235A0083587F201B6A1A68C9
:1013A00082431A6018688022024311431960704713
:1013B000004870470100040000B58C235A00835890
:1013C0001B6A002902D10349596200BD02485862D4
:1013D000FBE7C04603000080FF030080F0B55746DE
:1013E0004E464546E0B48C268A787300C3580F25D4
:1013F00015406F00D40958684A793E190C79814626
:10140000120218682243F5004519101C77003F307E
:101410003F26B043CC7882460320160420400128A2
:1014200032D01C69A402200C80468024E00544468A
:10143000204330432860FC001869A446CC44041CB7
:10144000604604604260186901378046D0444446D3
:101450001C61C97803200140012920D019698C0240
:10146000210C8024E40521430E436E601869FE00C0
:101470004E44306072601A695546AF181F611CBC3B
:1014800090469946A246F0BD18698002040CA04619
:101490008820C4054046044334432C60CBE71869D8
:1014A00088248102090CDDE77047C04630B58C24E2
:1014B0006300C258802510680F220A4029400B1C87
:1014C0005D1EAB415400E418E300C3181C680A48D1
:1014D00004401C60002A09D0002908D15A688021E4
:1014E0000D0610402C4305431C605D6030BD5968FB
:1014F00008405860FAE7C046FFFFFFBF00B58C22E6
:101500005300C2580F20084010D0D3684000136128
:101510000B06D90F12684318D800131819688022D7
:10152000D0050143196059680843586000BDC046A2
:1015300030B58C225300C4580F220A402568500051
:101540000B0616D50130C300EB185D681A680A490E
:10155000246A0A4029401A6059600125A46985401F
:101560002C4201D004330A1C802041050A431A6032
:1015700030BD1301E8E7C046FFFFFFDF70B58C22E6
:10158000540080230F220A40194000590D1C6B1E85
:101590009D41540006686519EB00F318002A07D135
:1015A0001A68002A1CDB8024A5052A431A6070BD36
:1015B0001E68002E21DB026A802085052E431E60F6
:1015C0004D1EA941D0696418E04001210142EED0CE
:1015D000586800281EDB8022940520435860E6E707
:1015E0000121A9400D1C016A4869284348614E69E0
:1015F0002E42FCD10D621A68D5E70122AA40151CC3
:10160000026A50692843506156692E42FCD1156226
:101610001E68D1E7A1400C1C5169214351615669F4
:101620002642FCD114625868D5E7C046F0B55F4643
:1016300056464D464446F0B48C24620082588023BE
:101640000F2455680C401940081C431E9841AB46B6
:101650006500281816684700C300BC46F318002C24
:101660003BD0204E5F681C68374034405F60BA460C
:10167000176A1C60BE690127B0463E1C864047467B
:10168000374201D0043354468027780504431C6058
:10169000002913D056690135EE400121314207D0AF
:1016A0008027380604431C605369A9408B4353616B
:1016B0003CBC90469946A246AB46F0BD0A4A6146FC
:1016C0001440CF005D461C60E81946688022310452
:1016D00015060D432C431C60EAE71968014E0E40C5
:1016E0001E60E5E7FFFFFFDFFFFF00FCF0B58C2584
:1016F0006C000059151F066A341C24340D2D09D9BD
:101700000120424237480025002B0DD125682A4090
:101710002260F0BD344FAD007F59BF468021334A6F
:101720000D060020002BF1D027683D432560F0E72F
:101730008020C5052E4A0020E6E7012252420025FE
:101740000020E1E70F250D400906341CCF0F6E0085
:10175000F11901268E40311C002D0ED1042A3CD0F7
:101760008026244A3502002B12D0C2691143C16180
:10177000002027683D432560CBE7002B0DD0C369CF
:1017800080251943C161042A24D0AD010020F0E76F
:10179000C3698B43C3610020B8E7C569F1430D40BD
:1017A000C561042A0CD0C569134B2940C161C169C8
:1017B000124E19404B1E99414A4232430020A5E780
:1017C000C2690F4F17407A1E97410E4A7842024372
:1017D00000209BE76D010020CBE780270A4AFD012E
:1017E000C1E7C046010004001C320000FFFFFF7F7C
:1017F000FFFFFFBFFF7FFFFFA8AAAAAAFFDFFFFF2F
:1018000054555555FFEFFFFFFFBFFFFF38B58C253F
:10181000031C0F2468001B580C400D066400E90FE0
:1018200065181868EC0004195D682368991C194351
:10183000880005D50A490B402360A3681940A160C0
:10184000A968101C082201F087FB6068830E9806C7
:101850006060A9688D022A0C10436060082038BDC2
:10186000FFFFFFDF00207047F0B55F4656464D464C
:101870004446F0B40F270F408C247B0066009B4643
:10188000802386590B409A46591E8B415B4434682D
:10189000716883B05D00D800A94624180191002F1B
:1018A00004D00125B1699D4029423ED16588019847
:1018B0004946AB05CD00451969689B0DC81A80469D
:1018C0002968101C424601F047FB21688A0E9306E6
:1018D0002360002F16D0306A51464A1E9141C769D5
:1018E0005944CF4001223A420CD08369B361B069B8
:1018F000C84002421DD04D460135019AE900636897
:10190000551804346A682F6880201604BD02020648
:101910003243290C0A4313434046236003B03CBCC6
:1019200090469946A246AB46F0BD01230434994443
:10193000BCE748460138019E043CC7002368F519FE
:10194000E0E7C046F0B55F4656464D464446F0B423
:1019500085B08C277E0001920F2780220A400F401D
:101960008659111C1D1C7B0099464B1E9941494408
:1019700034687368C800904624184A000293002F08
:1019800030D1211C08390868802382461806534646
:10199000184308602068029B810E8906D2002160EE
:1019A0009B18AD051868AD0D2A0494468202120CEE
:1019B0006046024311432160186801992A1C01F016
:1019C000CBFA23689A0001D5002F1ED180210E0684
:1019D00033432360281C05B03CBC90469946A24680
:1019E000AB46F0BD336AD8699A46031CCB40012050
:1019F00084461842CED053469869031CCB406046BB
:101A00001842C7D004340132C4E74346591E8B4103
:101A10004B44012277699A40141C3C437461D9E716
:101A2000F8B58C2254000459051CEA230020E85420
:101A3000266AA06160612068B060A768F760E92746
:101A4000E95D66680A01002101F08AFAEA5D002179
:101A50001201606801F084FAF023EB58A168D8798C
:101A6000890222680004090C01431160A1683160F9
:101A7000D8797060A16840318802D979000C0904D6
:101A800001435160A06808214030B060F160A06857
:101A9000DB7980021904030C0B439360A06830616A
:101AA000EB5D012B0AD980210C320423CE05E920FD
:101AB00040C2295C01338F009F42F9D8E168266A51
:101AC0002161074A074C084B0027B7617761F26133
:101AD000346273623068802505433560F8BDC046C6
:101AE000FF030000FF0300C0FF030080F0B55F4666
:101AF00056464D464446F0B45668137985B0029078
:101B00008946141C0196002B07D0744805B03CBCD4
:101B100090469946A246AB46F0BD117B08014A01AA
:101B200036189046B246D044121847462837151C3E
:101B300067602835BB0707D04746BA1A013203232E
:101B4000571901353B42FBD1B6214E00BA196260EC
:101B5000381C4946221C01F061F900212822404628
:101B600001F0FEF98C20424621684300019857623B
:101B7000FA5053465360116210606268AE190391C7
:101B8000131C910607D06C3AFF3A551B3F22AB1944
:101B900001361A42FBD14046836080336360C360E4
:101BA0004B469D682A78A846002A76D000230F2548
:101BB0003F21B4469B464646A946B8468A46271C5E
:101BC000331C00200096002A15D0191C1A784C7876
:101BD0009B18052CF7D18C783D7B4E463440A542AE
:101BE00059DD4E790C7935022C433F3451468C43F4
:101BF0000019002AE9D1009E834500D28346F3787C
:101C0000B2781802104336183278002AD8D15946D3
:101C10003C1C664647464B008036F618A3689E4239
:101C200000D972E7019A9D1BB0186060A560BC6D79
:101C3000002C4FD0FB6D002B49D03C6E002C43D0C4
:101C4000786E00283DD0BE6E002E37D0F96E002988
:101C500031D03D6F002D2BD07A6F002A25D0BB6F7D
:101C6000002B1FD0FC6F002C19D0039E0023336083
:101C7000381CFFF7D5FE8C2250003D587F212E6A7C
:101C80000298346880228C43346033681A4332608F
:101C9000076000203AE7124838E70023BCE7114DFF
:101CA000FD67E2E70F49B967DCE70E4E7E67D6E7CE
:101CB0000C483867D0E70B4CFC66CAE7094BBB669B
:101CC000C4E7084A7A66BEE7064D3D66B8E70549AF
:101CD000F965B2E7034EBE65ACE7C0460A000400F2
:101CE0000900040009130000F8B55F4656464D464A
:101CF0004446F0B4061C8C204300F7583B6A1A6A2D
:101D00001A62596A5C680A40904600D578E063041C
:101D1000180F44468246A5053FD0E922B25C002A4E
:101D20003BD0351C0120E9215835002481468B46E3
:101D300018E0386A802102684800024249D15046C2
:101D4000092803D1F969194200D094E00222A96A56
:101D50002B68301C98475A46B25C01340435510058
:101D6000A1421AD94B46A34041461942F5D04A46F2
:101D70002242DED05046092803D1F969194200D029
:101D800071E0A96A2B680322301C98475846325CE0
:101D9000013404355100A142E4D847467A0004D505
:101DA000736B002B01D0301C9847F36B002B0AD0CB
:101DB00055460A2D04D80124354AAC40144202D1BC
:101DC000301C514698473CBC90469946A246AB46CB
:101DD000F8BD3B682F481A68996802401A600840AD
:101DE00080229860B158B36D0122301C9847386A40
:101DF0008023026859000A4302605B46F25CACE74C
:101E000080221D68D20415421ED180214A04154249
:101E100008D0186802431A60B36B002B02D0301C44
:101E20000021984780239B041D4200D16FE73A6A46
:101E300011680B431360A90325D4336B002B00D129
:101E400065E7301C984762E71C68301C22431A6023
:101E5000FFF7E6FD301C00F053FFB36A002BB2D051
:101E6000301C9847AFE70522A96A2B68301C9847B9
:101E70005A46B25C71E72B680422A96A301C984765
:101E80005B46F25C69E7F36A002BDAD13FE7C046B4
:101E900001060000FFFFFFDF38B5051C4878232846
:101EA00001D9214838BD214C8000205887460020A8
:101EB000002BF7D02C6A002CF4D01168281C1A1CB7
:101EC000A047EFE70020002BECD0AC6A002CE9D053
:101ED0008878C978126809020143281CA047E1E705
:101EE0002B6B0020002BDDD0CC788A7821021143A7
:101EF000281C9847D6E7002B12D0EB6B0020002B54
:101F0000D0D0291C1031281C9847CBE76B6B0020E0
:101F1000002BE9D1C6E7AB6B0020002BE4D1C1E771
:101F2000103515600020BDE70200040054320000A7
:101F300070B5051C012A2CD0022A02D0344C201C7A
:101F400070BDB2267400035D7F221340212BF5D1B2
:101F5000B4225300C35C087E984202D04C7E9C425F
:101F6000ECD1B5208E2672004300AC58EB5AB22655
:101F7000E01AA85074008E222E1950004C6C2A18BA
:101F8000081C311CA047041ED9D1281C00F02CFFCE
:101F9000D5E7B2204300EB5C7F221A40212ACDD145
:101FA000B4225600AA5D0C7E944202D0487E904234
:101FB000C4D1922460008E222C185600AC51DB094B
:101FC00012D1B22674008E202B1942004E6C081CD0
:101FD000AA18191C0023B047041EB0D1B522530023
:101FE000E95A0029ABD1D0E7B22046008E249023D5
:101FF00062005800AE190C6C2B18AA18081C311C72
:10200000A047041E9BD1281C00F0C2FE97E7C046E3
:102010000200040038B54C78032C0CD0212C13D0CE
:10202000012C01D00F4838BD446A002C03D0111C8C
:102030001A1CA047F7E7C46A002C0BD08D78C9782A
:1020400009022943A047EEE71030106007221A80EA
:102050000020E8E710680021402200F081FF002006
:10206000E1E7C0460200040008B5A1230371002384
:1020700041718371C371037243728372C372012908
:1020800009D0002903D020290ED00B480BE0002AEC
:1020900001D0012181710368017F021D181C0823F2
:1020A000FFF750FC002008BD02730223120A83725E
:1020B00042730148F7E7C046030001004C20704717
:1020C000F8B54F464646C0B40D68071C0C1C904638
:1020D0008E684B68A90703D0472B01D8474825E0F5
:1020E000281C03224B30483B93439043206063609D
:1020F00000214822281C00F033FF41494148236A4F
:10210000626A29646864A16AE06A2B626A62236B6E
:10211000626BA962E862A16BE06B2F602B636A635C
:10212000A963E8637378042B04D037480CBC90464D
:102130009946F8BD7379022BF7D131790129F4D88A
:10214000B07828763279012A1AD0E36859780429C0
:10215000EBD15A790A2AE8D198790028E5D19A7802
:102160006A7619781E795A18B146484529D21178ED
:10217000161C8C4671786244052916D00130F4E7AC
:102180003378F618331C31785A787618052A06D039
:10219000042AF7D1287F0028D7D11C48C6E7DA786F
:1021A000032AEFD19E782E77F4E7F1780229E5D162
:1021B000B1784EB2002E16DBE9761E790130B146B9
:1021C000D3E7AB7E002BE8D0E87E0028E5D0616C39
:1021D000381C00290CD02A1C00F094FE0C4F6764B8
:1021E00044462560A2E7A976197901308946BCE703
:1021F00007492A1C00F086FEF2E7C0460A000400E8
:1022000015200000991E00000800040009000400C9
:10221000311F000000B5B2225100435CDA0601D044
:10222000044800BD011C8E22ED315300C150002036
:10223000F7E7C046010004007047C0467047C0463B
:1022400000B5B2235A00815CCB06DB0E012B30D0E7
:10225000022B0AD0002B01D0214800BD011C8E2387
:10226000EE315A0081500020F7E7B4214B00C35CE7
:102270008F22134080221A422BD101219940ED2256
:10228000825C002A01D11A07E6D182235A008358C2
:102290000B42E1D084235A008358922219404B1EEE
:1022A00099415300C152C1188E235A008150002019
:1022B000D3E7ED22815C0029CED0B4235900EB2274
:1022C000415C835C9942C7D2922100224B00C252EA
:1022D000E9E70F21194052028A40111CCFE7C0469E
:1022E0000100040030B5B2246100031C405CC2064A
:1022F00007D1414D5A5D022A05D0032A38D0012A60
:1023000060D03E4830BDB320FC2245009A585C5D49
:102310001178002C22D0601E01250540002963D1D0
:102320000120A0421AD0002D04D000290DD1013087
:10233000A04213D0002905D0D1789578090229430D
:102340005218117801300029F1D0D178957809021E
:102350002943521801301178A042EBD10029D0D086
:102360008E2568001A509478D278110221432FE00C
:10237000B3225400F42159581C5D0A78002C1AD05D
:10238000601E01250540002A2BD10120A04212D059
:10239000002D04D0002A09D10130A0420BD0002A20
:1023A00001D089180A780130002AF5D08918013047
:1023B0000A78A042F3D1002AA3D08E246500595197
:1023C000097805E0F0248E2118594A00985012210E
:1023D000902252009D5A00208D4200D892E79952D7
:1023E00090E789180A78D0E7D178907809020143FC
:1023F0005218117894E7C0466701000001000400FC
:1024000000B5B2235900435C1F221340012B01D0B9
:102410000A4800BDED21425C002AF9D0B4225300E5
:10242000EB21C35C425C9A42F2D91133FF338E2216
:10243000C318510043500020EBE7C04601000400E0
:10244000F0B55F4656464D464446F0B4B2246200AD
:10245000815C051CC80685B0C30E012B08D0534E05
:10246000301C05B03CBC90469946A246AB46F0BD38
:10247000ED27EE5D002EF2D0EA202B5C012B73D00D
:10248000F8242C590022B421B32300279246480097
:102490005A00464E0297B946804600279346227856
:1024A000002ADDD06378042B3FD0052B0ED0022B01
:1024B00001D0A418F3E7ED2160796B5C9842F8D065
:1024C000E378A278180210432418E8E74346E95C51
:1024D000B942EED1A3788F211940802001910842A2
:1024E0003BD10120884003905B46E95C49453ED0E2
:1024F00002988145DDD103994846534602900B422C
:10250000D7D1CA4382214B00E85884211040E850BB
:1025100048002B5801991A402A50281CFEF7EEFF5C
:10252000227849460291A418B9E7E07843468146EB
:10253000A778E85C00218A468742BAD15B46E95C0D
:102540008945B6D1E8191130FF3002784E46067041
:10255000029222780026A418A1E70F2080230840C9
:10256000590281400391BFE7FC216C588AE7822120
:102570004B00EA58039984200A43EA504300EA5882
:10258000281C8A43EA50211CFEF728FF281C0199C9
:10259000FEF78CFF281C0199FEF7CAFF03985246EC
:1025A000024392462278A41879E7C046010004004D
:1025B000F8B55F4656464D464446F0B4B222510047
:1025C000041C405CC30628D1B3267500635D002B54
:1025D0002AD0EA23E75C012F00D105E1F8256559EF
:1025E000002680228221B24693464F002A78002A94
:1025F0000BD06B78042B00D18AE0052B67D0022B1F
:1026000059D0AD182A78002AF3D1B3204600ED2125
:10261000655CA45D0020A54200D075483CBC904696
:102620009946A246AB46F8BDED26A355E925675D60
:10263000012F28D980238222590201255600012723
:10264000884608E04146A940194212D1E922A35C1C
:1026500001359D4217D2381CA359A8400342F1D03E
:10266000291C201CFEF74AFF4146A359A9401942E4
:10267000ECD080212943201CFEF740FFE922A35C17
:1026800001359D42E7D35B4A8227842186267B0061
:102690000025480077002550E551201CE25000211C
:1026A000FEF78AFEB3204600ED21655CA45D0020A4
:1026B000A542B2D1B2E7B3214B006879E35C834213
:1026C0002AD0EE78A87833020343ED188EE75346FC
:1026D000002B96D1AE788F2006405A46324278D0F1
:1026E0000F2380223340510299400B1CE059291CD2
:1026F0000343E351201CFEF771FE201C311CFEF742
:10270000D5FE201C311CFEF713FF2A78AD1879E79F
:10271000E978AD188A4675E7ED2163542879EB23F3
:1027200088263549E05472000023A354892063545D
:10273000324A8A2146004800A355A354304E235400
:102740008B2230485100A3556354E9262354A25DDF
:10275000012A26D9802001264202B046914608E08F
:102760004A46B2401A4212D1E920235C01369E4209
:1027700017D24146E359B1400B42F1D0201C311C25
:10278000FEF7BCFE4A46E359B2401A42ECD0594625
:102790003143201CFEF7B2FEE920235C01369E4245
:1027A000E7D314498426862200237000E1515100AA
:1027B00023506350201C0121FEF7FEFDEE797206C6
:1027C0000AD5EE23E05A01220243E2522A78AD18DC
:1027D00018E70123B34089E7EE22A65A01218E4370
:1027E000A6522A78AD180DE7FC202558F8E6C04619
:1027F00001000400010001001101000013010000AC
:10280000150100001701000070B5B2220D1C510027
:10281000041C405CC306DB0E08D1B3235E00A35B3F
:10282000012B37D0022B4AD02D4870BD022BFBD193
:10283000B4225000235C8F21194080230B4223D106
:1028400001268E40ED22A05C0028EDD00B07EBD0D6
:102850008222500023583342E6D0B3225000235A3C
:10286000002BE1D1002D30D18623580022580020C2
:102870003242DAD1201CFEF7D9FE84204200A15852
:10288000281CB143A150D0E70F260E405B02B34095
:102890001E1CD7E7236C002B02D0201C291C984754
:1028A000EE23002D05D0E05A02250543E552002015
:1028B000BBE7E25A02218A43E2520020B5E7094E03
:1028C000201CA15DFEF774FDAFE7201CFEF756FE4D
:1028D00084235D00615900200E436651A5E7C04680
:1028E0000100040069010000F0B5474680B4B22140
:1028F000041C4800265C7F239E4349D190277F001B
:10290000E25B0025002A03D1281C04BC9046F0BDE0
:102910008E20450062590021201CFEF7A5FF635957
:102920001A186251E15B0D1AABB2E353351C002B50
:10293000EAD1E823E25C002A11D0271C224DA837F7
:10294000984608CF002B07D0F969201C022298472F
:10295000A84226D14146625C01369642F1D3B223A9
:102960005D00675D60221740402F07D1A368002BF0
:1029700004D0201C0121984700281DD0201C802154
:10298000FEF7FCFD902000254300E5520025BBE743
:10299000922671006218201C0021FEF765FF0025B9
:1029A000B2E7051EB0D0201C8021FEF7E7FD902283
:1029B00000265700E653A7E7201C802100220023B1
:1029C000FEF7C0FF00259FE702000400F0B5474670
:1029D00080B4041C072A31D84A48920083589F4685
:1029E000E823E25C002A13D0261C474FA8360025B6
:1029F000984608CE002B08D0F169201C0322984786
:102A0000B84200D069E04146625C01359542F0D39E
:102A100090204600A25B4023402A00D8131C8E2041
:102A2000450062598021201CFEF78CFF66599021D9
:102A300033184F006351E25B101AE053002004BCCE
:102A40009046F0BD201C8021FEF7F0FDF6E72568DA
:102A5000201CA847F2E76668201CB047EEE7B222C8
:102A60005700E05D7F239843BAD1EC22A15C4FB2BE
:102A7000002FE3DA1940A154201CFEF78BFCDDE7A0
:102A8000E821625C002A13D0261CE8231E4FA836DA
:102A90000025984608CE002B07D0F169201C04229F
:102AA0009847B84219D14046225C01359542F1D38E
:102AB000B2256B00E15CCA091AD18E2190274A0029
:102AC0007E00A258A35B201C0021FEF7CBFEB5E7D9
:102AD000201C0021FEF7AAFDB0E70028AED0201C84
:102AE00080219026FEF74AFD00257300E552A5E7F8
:102AF0008E235D006259201C00210023FEF7B2FEE8
:102B00009CE7C046E432000002000400F0B54746EE
:102B100080B4061CB2204300F2180021301CFEF7DE
:102B200075FEB2225700F55D301CE909B524FEF7A9
:102B3000BBFC6100725A90204300F252E823F25C21
:102B4000002A12D0351C6B4FA8350024984608CDBA
:102B5000002B07D0E969301C01229847B84219D1EF
:102B60004146725C01349442F1D3B2277D00735D1B
:102B70005C06A30F19D0022B1FD0301C8021FEF75A
:102B8000FDFC902100224D0072530024201C04BC47
:102B90009046F0BD041EF9D0301C8021FEF7EEFCFB
:102BA000902200255700F553F0E7534C335D0B2B73
:102BB000E3D8524998000B589F46B368002BDCD0ED
:102BC000301C01219847041ED7D1B5214B00F05A83
:102BD000002800D187E0775DFD09D7D09020420022
:102BE000B25A4023402A00D8131C8E204500725947
:102BF0008021301CFEF7A6FE715990270A187B0031
:102C00007251F55A291AF152C0E7346A301CA047B4
:102C1000041EB2D10023301C80210022FEF792FE58
:102C2000B36C002BB2D0301C9847AFE7F269301C70
:102C30009047041EA1D1D1E7B769301CB847041EE4
:102C400000D09AE70023301C80210022FEF77AFE94
:102C5000736C002BE7D199E77569301CA847041EF7
:102C600000D08AE7BAE7301C002188E73169301CC0
:102C70008847041E00D080E7B0E7B2204300F45C30
:102C8000E20600D079E7B3235C00375D8022514231
:102C90003943EC257155301C802100220023FEF7BA
:102CA00051FE002472E7726A301C01219047041E15
:102CB00000D062E70023301C80210022FEF742FE94
:102CC000F36C002BAFD161E7776A301C0021B84765
:102CD000041E00D051E7EDE7F568301CA847041E3C
:102CE00000D04AE77AE7301C802100220023FEF75B
:102CF00029FE4BE7020004006501000004330000D8
:102D0000F0B5474680B40124EE23C452EC210023E1
:102D1000061C4354ED2033548222174D8424862010
:102D20005700610042007350B350F551E823F25C44
:102D3000002A12D0351C114FA8350024984608CD22
:102D4000002B07D0E969301C0E229847B84207D102
:102D50004246B25C01349442F1D304BC9046F0BDCB
:102D60000028FAD0301C8021FEF708FC90200025B6
:102D70004700F553F1E7C0460100010002000400DE
:102D800008B5B2214B00C2180021FEF73FFD08BD77
:102D900038B5041C90204300E25A4023402A00D852
:102DA000131C8E2045006259201C8021FEF7CAFDAD
:102DB00062599023111861515D00625B111A6153D1
:102DC00038BDC04638B5041C8E2045006259201C11
:102DD0000021FEF749FD62599021131863514B0001
:102DE000E25A101AE05238BD08B5802100220023B3
:102DF000FEF7A8FD08BDC04608B592214B00C218D9
:102E00000021FEF731FD08BD10B58021041CFEF73E
:102E1000B5FB902000224300E25210BD70B5B623EE
:102E2000151C0E1C5A000021041C00F099F82B7B85
:102E3000E922A354274A8021A2656450002B02D0C6
:102E40008420E26524502449244B2548254A2160EA
:102E5000E3602549254B6060626221612448A361DB
:102E6000244A2549EB6B6061E2612162002B29D085
:102E700023652B6C002B2AD06A6A29696365AB6ACB
:102E80002264A162AA69E96A6869A3632B6A226362
:102E9000E1636A6B3168E0626363286BF023AD6BBA
:102EA000A264E1507268B1686064E564F420F825BA
:102EB00022506151F068356980225600FC23A551EB
:102EC000E05070BD0D4B23652B6C002BD4D10C4B07
:102ED000D2E7C046CD2900000D2B000041220000A2
:102EE000E928000009280000E5220000B1250000C3
:102EF00015220000012400004124000039220000B6
:102F00003D22000030B5E824035D072B01D90748B6
:102F100030BD1D1C2A35AD0029501D1C3235A900BD
:102F200001330A5003550020F2E7C0460B000400AD
:102F300010B5E924045D64008C4201D2054810BD3F
:102F40000C1C16342031A400890022500B500020A4
:102F5000F5E7C0460300010008B500F06CF808BDB5
:102F600008B500F07EF808BD10B5431C820706D0F6
:102F70000130421E1278002AF8D1C01A18E0026807
:102F80000C490D4C51189143214201D10430F6E710
:102F9000D4B2411C002C0AD0FF242402811C2242FE
:102FA00005D0FF242404C11C224200D0011DC81AF0
:102FB00010BDC046FFFEFEFE8080808003000B43F4
:102FC00021D4002931D00122D207030901E00901EF
:102FD00012099942FBD9430801E04900520899427D
:102FE000FBD900E04908401A07D35241FAD3014601
:102FF0001046704749084018F7D29218FAD3401883
:10300000014610467047CB0F00D04942021000D550
:103010004042534008B5FFF7D4FF0CBC521000D318
:103020004042002A00D549421847F446002000F0EB
:1030300001F8604770478446830708D18B0706D1A3
:10304000131F04D304C904C0043BFBD21A1D52420F
:1030500005D0891A801A8B5C83540132FBD16046FB
:1030600070478446043A09D3830707D109060B0A3F
:1030700019430B0C1943043A02C0FCD2043203D0AA
:1030800001700130013AFBD1604670478C46411E09
:103090007144095A49008E4461467047040309048B
:1030A0000E03430041004E00410041004E00240346
:1030B00055005300420032004900490043002000FF
:1030C00043006F006E0076006500720074006500BA
:1030D0007200120332003000310034003100310040
:1030E00032003200060334003000000012010002FA
:1030F000EF020140F129F2330001010203014155C1
:10310000432D3230313531323038000094310000F7
:10311000F03100000000000000000000000000008E
:10312000103200000000000001112202001BB70055
:103130000001010000020100000301000004010081
:103140000005010000060100000B01010012010052
:103150000013010000000000C027090090051000C6
:10316000C05C1500F0B31A00200B2000009F240063
:10317000E0322900C0C62D0050973100E0673500CD
:103180007038390000093D0040164000802343009C
:10319000C030460011130000ED1A00002513000096
:1031A000E91C0000211A00000D1300006D1300003F
:1031B00095130000B9130000DD130000A9140000EE
:1031C000AD140000FD140000311500007D15000055
:1031D0002D160000B11300006918000065180000EA
:1031E0000D180000451900004D130000ED160000F9
:1031F000052F0000312F0000812D0000912D0000CF
:10320000C52D0000E92D0000F92D0000092E000059
:10321000BD200000C120000069200000441700000C
:1032200044170000001700000017000000170000FE
:103230000017000000170000001700000017000032
:10324000001700003A170000301700001C1700009C
:103250003A170000AE1E0000A21E0000C41E0000AF
:10326000A21E0000E01E0000A21E0000A21E000020
:10327000A21E0000A21E0000A21E0000A21E00004E
:10328000A21E0000A21E0000A21E0000A21E00003E
:10329000A21E0000A21E0000A21E0000A21E00002E
:1032A000A21E0000A21E0000A21E0000A21E00001E
:1032B000A21E0000A21E0000A21E0000A21E00000E
:1032C000A21E0000A21E0000A21E0000A21E0000FE
:1032D000A21E0000F61E0000A21E00000C1F00002F
:1032E000161F00003C2A00004E2A0000562A00004B
:1032F0005E2A0000802A00003C2A0000D02A00003C
:10330000442A0000D82C0000C82C00007A2B0000B2
:10331000A62C00007A2B00007A2C00006C2C0000F8
:10332000662C0000582C0000382C00002C2C0000CB
:043330000A2C000063
:1033340009024B00020100C0FA080B000202FE0061
:1033440004090400000102FE000405240010010524
:103354002401010104240202052406000107058258
:103364000310000209040100020A00000407050119
:103374000240000007058102400000008025000093
:103384000C31000000000040050000007510000032
:103394000000000000000000000000000000000029
:0400000300000117E1
:00000001FF
